:1000000012C02CC02BC02AC029C028C027C026C0BF
:1000100025C025C023C022C021C020C01FC01EC0D3
:100020001DC01CC01BC011241FBECFE5D4E0DEBF25
:10003000CDBF10E0A0E6B0E0E6E6F6E002C0059035
:100040000D92A036B107D9F710E0A0E6B0E001C0EC
:100050001D92AD36B107E1F7C5D103C3D1CF1F92D1
:100060000F920FB60F9211242F933F936F937F93AC
:100070008F939F9385B38F6085BB98B19072809169
:1000800060009817E1F480916100853028F4809138
:1000900061008F5F8093610080916100823089F4FC
:1000A000809163008F5F809363008091630084364A
:1000B00041F481E0809362001092630002C01092CC
:1000C00061009093600080916C00882311F031E012
:1000D00009C082B390E026E0969587952A95E1F7CE
:1000E000382F317080916500882309F05FC020911E
:1000F000690086B390E080729070880F991F880F16
:10010000991F282B209369002091690086B390E005
:100110008870907063E0880F991F6A95E1F7282B2B
:100120002093690082B3807C82BB80916700853018
:1001300028F0332319F085B38E7085BB809167005A
:100140008A3028F0332319F085B38D7085BB8091F8
:1001500067008F3028F0332319F085B38B7085BB8F
:1001600080916700843128F0332319F085B38770BC
:1001700085BB909A9091690080916A00981791F4DC
:1001800080916B008A3021F480916900809368002F
:1001900080916B008F3F41F080916B008F5F809367
:1001A0006B0002C010926B0081E029C08091650055
:1001B000813041F58091670065E047D282B3807C51
:1001C00082BB9923D1F0332319F085B38E7085BBA0
:1001D000913061F0332319F085B38D7085BB933076
:1001E00028F0332319F085B38B7085BB943029F444
:1001F000332319F085B3877085BB919A82E0809391
:100200006500CAC080916500823009F582B3807CA8
:1002100082BB809166008D3228F0332319F085B3BC
:100220008E7085BB80916600823328F0332319F0ED
:1002300085B38D7085BB80916600873328F03323AA
:1002400019F085B38B7085BB929A83E0D8CF8091EB
:100250006500833051F582B3807C82BB809166005B
:10026000893128F0332319F085B38E7085BB8091D6
:1002700066008E3128F0332319F085B38D7085BB6D
:1002800080916600833228F0332319F085B38B7098
:1002900085BB80916600883228F0332319F085B33E
:1002A000877085BB939A84E0AACF809165008430E3
:1002B000C9F58091690080936A0086B390E08873E5
:1002C000907023E0959587952A95E1F780936900D2
:1002D00082B3807C82BB80916600853028F0332316
:1002E00019F085B38E7085BB809166008A3028F046
:1002F000332319F085B38D7085BB809166008F30F4
:1003000028F0332319F085B38B7085BB809166008C
:10031000843128F0332319F085B3877085BB949A14
:1003200085E06DCF809165008530B0F190916900D6
:1003300086B38873892B809369008091660065E09D
:1003400084D182B3807C82BB9923D1F0332319F00E
:1003500085B38E7085BB913061F0332319F085B37E
:100360008D7085BB933028F0332319F085B38B70E3
:1003700085BB943029F4332319F085B3877085BB8E
:10038000959A1092650080916200882329F081E09F
:1003900080936400109262009F918F917F916F9182
:1003A0003F912F910F900FBE0F901F90189583E0F3
:1003B00087BB8FE084BB8FE781BB82E083BF89B7B7
:1003C000816089BF8EE890E09BBD8ABD87E490E0A4
:1003D00099BD88BD80E18FBD8AE08EBD80E488B97B
:1003E00078940895FF920F931F9383E087BB8FE06B
:1003F00084BB8FE781BB82E083BF89B7816089BFFF
:100400008EE890E09BBD8ABD87E490E099BD88BDF1
:1004100080E18FBD8AE08EBD80E488B9789460E089
:1004200090E040E02BE338E1F0E0E0E070E050E005
:10043000B0E0A0E000E414E0F12E11E0809164004F
:10044000882309F44BC090FD47C04F5F4C3389F5BA
:1004500080916C00882369F1383149F42B3311F411
:1004600020E003C0222319F421E030E005C02F5F13
:100470002C3311F43F5F20E0C09B07C0E31729F441
:10048000F21719F4992309F4B1E0C19B11C0531775
:1004900079F4721711F0352F0BC0992321F0272F13
:1004A000352F40E00CC0272F352F40E0A1E003C0DE
:1004B00040E0992321F4209366003093670082B3D3
:1004C000802782BBBB2311F4AA2321F087B38F2599
:1004D00087BB02C0BA99BA981092640080916800F4
:1004E000861709F4ABCF992371F5662361F58091E6
:1004F0006800843029F4969810936C0091E023C032
:1005000080916800823039F4F0936600E0936700D0
:10051000C09A92E018C080916800813039F47093DD
:10052000660050936700C19A94E00DC08091680006
:10053000803119F4C098B0E006C08091680088301E
:1005400011F4C198A0E08091680082FD08C090FF7E
:1005500006C0209166003091670090E040E08091F5
:10056000680081FD10C091FF0EC0F0916600E0911F
:1005700067002093660030936700FF2319F4EE2391
:1005800009F4C09890E08091680080FD10C092FF4F
:100590000EC0709166005091670020936600309302
:1005A0006700772319F4552309F4C19890E08091EE
:1005B0006800807E803409F59923F9F08091660007
:1005C0008B3330F4809166008F5F8093660007C0A4
:1005D00010926600809167008F5F80936700809122
:1005E0006700883121F480916600882321F480918E
:1005F0006700893110F01092670080916800807E5A
:100600008038A9F4992399F0809167008F5F8093D7
:10061000670080916700883121F48091660088230B
:1006200021F480916700893110F010926700809169
:100630006800807E803231F4992321F010926700A7
:100640001092660060916800F9CE991B79E004C0B1
:10065000991F961708F0961B881F7A95C9F7809501
:060660000895F894FFCF9D
:00000001FF
